:1000000080710010C1010000C5010000C70100009F
:10001000C9010000CB010000CD010000D283FFEF39
:10002000000000000000000000000000CF01000000
:10003000D101000000000000D3010000F901000020
:10004000D7010000D7010000D7010000D701000050
:10005000D7010000D7010000D7010000D701000040
:10006000D7010000D7010000D7010000D701000030
:10007000D7010000D7010000D7010000D701000020
:10008000D7010000D7010000D7010000D701000010
:10009000D7010000D7010000D7010000D701000000
:1000A000D7270000D7010000D7010000D7010000CA
:1000B000D7010000D7010000D7010000D7010000E0
:1000C000D7010000D7010000D701000000F002F8BE
:1000D00000F03EF80AA090E8000C82448344AAF1A4
:1000E0000107DA4501D100F033F8AFF2090EBAE8A2
:1000F0000F0013F0010F18BFFB1A43F0010318475C
:10010000CC530000EC530000103A24BF78C878C1EB
:10011000FAD8520724BF30C830C144BF04680C600D
:10012000704700000023002400250026103A28BF55
:1001300078C1FBD8520728BF30C148BF0B60704759
:100140001FB59DE8030004F014FE1FBD10B510BDDF
:1001500004F045FE1146FFF7F3FF00F0D8FB04F072
:1001600063FE03B4FFF7F2FF03BC04F093FE00004C
:10017000D0F800D0D0F804F070B500230E4D0AE09E
:10018000CE5C04885B1C86EA14269BB235F81660A8
:1001900086EA04240480521E92B2F1D270BD30B5BA
:1001A000064C0022855CA35C521C1D4492B2CD54C7
:1001B000FF2AF7D930BD0000E04F0000E04E0000FC
:1001C00008480047FEE7FEE7FEE7FEE7FEE7FEE73A
:1001D000FEE7FEE7FEE7FEE703480449044A054B55
:1001E00070470000CD0000008021001080710010D9
:1001F000806100108061001009480168491C01609D
:1002000001680068704707480221416000210167CA
:1002100041610B22C260C16301214160002070472F
:10022000DC00001000000940EFF3108010F0010F17
:1002300072B64FF080404FF0000202704FF0AA03F8
:1002400003724FF05504047202614FF0FF024260E6
:100250004FF0030202700372047200D162B6FEE72F
:1002600019480421016107210160002141614162B7
:1002700002214160C168C906FCD400E08168C16800
:100280004907FBD4002070470F498860C868C00642
:10029000FCD48868704700B50B46024604E000BFF6
:1002A00012F8010BFFF7F0FF5B1EF9D200BD00B59D
:1002B0000B46024604E00020FFF7E6FF02F8010BC0
:1002C0005B1EF8D200BD00000080084010B591FB15
:1002D000F2F491FBF2F302FB1411C0E9003110BDFE
:1002E0007047704770470000004870472421001095
:1002F00070477047004870471C210010FFFFFFFF48
:1003000070B5284C607820B30026274D012810D006
:1003100002280DD1A8686168401A2449884215D383
:100320002348406B400011D5012002F02EF9667081
:1003300070BDA8686168401A1E498842F8D3002041
:1003400002F023F9A86860600220607026700C201B
:1003500005E020780028EBD1012020700D20BDE8B9
:10036000704001F09BB9002802D10E49012048706D
:10037000704710B501F026FE0A490020487010BDF4
:1003800008480121417008498968416070477047F9
:100390007047022803D0032803D100F032BE00F0DA
:1003A0004DBE70470C01001000000940A0860100FE
:1003B00000C0092040420F0000210160C0E9011087
:1003C000704710207047034640688C46002818BFCD
:1003D00088423CBF03464068F8D3186818448842F6
:1003E00007D00CF1030020F00700001D411A521A3B
:1003F0000146081D0A6004F008BC704700000000B8
:10040000000000008C0C0000FB4910B5486D000591
:100410000CD4FA4A906843F698239468241A9C42B4
:10042000FBD3486D000501D4012010BD052001F06B
:1004300035F9002010BD70B5F04CA668042001F01D
:100440002DF9EF4D03E000BFFFF7DEFF48B1A068D4
:10045000801BA842F8D308E0FFF7D6FF08B10120BF
:1004600070BDA068801BA842F6D3002070BD2DE9A6
:10047000F041092001F012F9E24800264FF47A77A2
:100480000670C821384601F0BFFADC4CA06842F281
:100490001075A168091AA942FBD3C821384601F09A
:1004A000B3FAA068A168091AA942FBD3C82138464B
:1004B00001F0AAFAD448022186708171C670BDE8A5
:1004C000F0818CB04FF00009CDF8289046208DF8CF
:1004D00014008DF8179037218DF81510DFF82CB324
:1004E0003821CDF824908DF81610DBF80020CA468C
:1004F0004FF6FF031A40C64B42F480721A43CBF802
:100500000020C449C448C84DC1F800A00068C349D0
:10051000A0F56C50FF380860C14900F5E050086054
:10052000C049400A0860F8202870FF206870A87051
:1005300001F002FAB44CBD4A002094F9051052F8BB
:1005400021202B1803F58053115C401C83F8001800
:100550006028F6D34FF4E175294640F2491001F0C6
:1005600053FA294640F29F1001F04EFA4FF400551D
:10057000207808B1FFF7C4FEA07938B1012819D05E
:1005800003287DD0207800287BD084E10A2001F068
:1005900085F800F08DFE002874D10120A0714FF481
:1005A000005584F803A0062001F078F80A2001F035
:1005B00075F884E1192229469D4800F039FE9C48CF
:1005C000007E002876D09A480078062871D2DFE8AD
:1005D00000F0C3030B72727540F204409449008826
:1005E00004904968814264D091484FF00109417AF2
:1005F00001295ED1D0F80A1019B98E498969C0F86D
:100600000A108B484FF00006007A400720D54FF4BF
:100610008078874F17E0072001F040F8A91942467B
:100620008548193100F004FE814983481931FFF7EC
:10063000B6FDD7F80A007E4930444246193100F031
:1006400079FF06F58076D7F80E00B042E3D823E0B4
:10065000DFF8DC811BE0072001F020F8D7F80E005E
:10066000B846871B402F00D94027A9193A4672483F
:10067000193100F0DDFDD8F80A003A46304402E0B6
:10068000F0E001E1EBE06C4900F054FF3E44D8F8A3
:100690000E004746B042DED86548017801295BD19B
:1006A0004FF0E0220906C2F88011D0F80A0000F0ED
:1006B0006FFF51E071E04FF0010950E05C484FF0EE
:1006C0000109417A03294AD153495C4A4FF0000697
:1006D0000B681360027A520720D54FF4807780466A
:1006E00017E0072000F0DAFFA9193A4652481931FD
:1006F00000F09EFD4E4950481931FFF750FD464825
:100700003A46006881194A48193000F080FD06F524
:100710008076D8F80E00B042E3D81DE0804616E09F
:10072000072000F0BBFFD7F80E00871B402F00D931
:100730004027A9193A464048193100F079FD36485A
:100740003A46006881193C4800F061FD3E44D8F803
:100750000E004746B042E3D83548007EE8B1344E3B
:10076000307AC00614D535484FF40051012201609B
:1007700005F1180104A8CDF810A000F039FD30787B
:1007800020B1C8214FF47A7001F03EF9307E20B1DB
:10079000307A800701D5FFF747FD25481B35D0F893
:1007A0000E000544224800F077FD18B302201549D9
:1007B000A0714FF4005581F800A00B2000F06EFFEF
:1007C000B9F1000F40D00D494FF000098A6842F29C
:1007D00010738868801A9842FBD34FF42F714FF43E
:1007E0007A7001F011F90448406D400528D50020C9
:1007F0000B9027E028E0000000C00920000009401D
:1008000080841E0068000010BC0000100CED00E0A9
:100810000000FA05AC000010B80000109C000010A9
:1008200094000010980000103902001060000010C1
:100830002001001020520000B11C0010B000001078
:100840000B9808B9FFF7F0FCE078401CC0B2E070EC
:100850000C2802D30120A07001E0A07878B3FFF744
:1008600006FE2CE04E4881680A98091A099800EBA8
:100870004002C2EBC010B1EBC00F20D300200A90A1
:10088000099084F806A01AE00120207001F0BCFE57
:10089000012001F07AFE4348007880B1002105A8CC
:1008A00000F018FC58B10320A0713D4884F803A063
:1008B0004FF4005580680A904FF47A7009903A4ED0
:1008C000706D00053FF554AE35488268374B81683E
:1008D000891A9942FBD3706D0005F3D4706D000541
:1008E000FCD42020B06532214FF47A7001F08CF8EE
:1008F000706B40000AD5DBF800102D4A01F4E0616E
:100900001143CBF80010BFF34F8FFEE7FEE7294CF1
:100910000025FF202560A580A571607100F05EFFB5
:1009200001F0A0F8FFF76FFC00F05CFE002000F083
:10093000B5FEFFF795FC1C48406B400013D51849E5
:1009400088681D4A8B681B1A9342FBD3FFF75CFD36
:1009500048B1FFF770FD30B1FFF76DFD18B1FFF73B
:100960006AFD00B1657100F035FC00F0A1FC80B1BA
:1009700000F015FE68B1022000F090FE94F9050029
:10098000401C03D10D48806900F002FE0120607018
:1009900004E0022000F082FE65706571FFF791FDB2
:1009A000000009406800001000C00920A086010076
:1009B0000400FA05BC00001020A10700205200002E
:1009C0002DE9F047FE4A00234FF40077156A4FF4F3
:1009D000FF79C5F30724DFF8ECA34FF4E05CDFF800
:1009E000E883FA4E25E0B84216D213280CD014281A
:1009F0000CD048450CD0A0F58072FF3A0AD03E28B2
:100A000013D81AF8002011E0EAB20FE022460DE0F8
:100A100055220BE0AA2209E0604506D208EB00024D
:100A2000A2F5805292F8002E00E00022F254401C01
:100A30005B1C8B42D7D3BDE8F08770B5E04D2C6BC3
:100A4000402C00D94024E86AE96902198A4202D997
:100A50000C1A042169702146FFF7B2FF2246DB49D8
:100A6000822001F08EFEE86A2044E862286B011BB8
:100A7000D74829638268A2EB0402826005D06978B6
:100A8000022901D00021017370BD03216970F9E7CB
:100A9000CF4910B5CF4808600D22822001F071FEC9
:100AA000C7490520487010BD70B50D46CA49496D4B
:100AB000490521D4B0F5007F1ED3C849C04CB0F51C
:100AC000E05F1AD28A68A369D21AC54B9A4204D34E
:100AD0008968A161002161606161BD4900235F39BE
:100AE000B94A07E0C4181444CE5CA4F580545B1CDA
:100AF00084F8006EAB42F5D370BD626922B98A6892
:100B0000A2618A686261A060B64A5279002AF3D174
:100B10008A686369D21AB44B9A421CD2B34B012241
:100B20001A708A68A26189686161A168401A616867
:100B3000884203D9616A884200D26060062000F0D2
:100B4000ADFD61682A46BDE87040A14801F500513D
:100B50005F3800F05CBBBDE870400C2000F09EBD2B
:100B600010B5974CA178E06A4218E1698A4206D92B
:100B7000081AA07005206070022001F0BDFDA17868
:100B8000E06AFFF791FFA178E06A0844E062206B19
:100B9000421A8F4822638368A3EB0101816002D06F
:100BA0006178052904D100210173BDE810406FE789
:100BB00010BD2DE9F041824CA178E06A4218E1694C
:100BC0008A4206D9081AA07005206070022001F040
:100BD00093FD7F4D0021A0787C4B5F3DE26A08E0E9
:100BE00056186F5C9E5DBE4202D00021A16202E0F9
:100BF000491C8142F4D31118E162216B0A1A74492D
:100C000022638B68A3EB0000886002D0607805281F
:100C100008D1A06A20B100200873BDE8F04137E791
:100C20000120F9E7BDE8F081694810B51F38D0F818
:100C30001110027D09BA21F0FF011143604A4902F7
:100C4000D162C18A49BA49021163806888420CD0D6
:100C5000822001F051FD022001F04EFD5C4902208E
:100C60000873FFF715FF002010BD012010BD70B5FF
:100C70005748574D1F380224816829B1007B000670
:100C800007D4022001F038FD2C73FFF701FF00208C
:100C900070BD012070BD10B54D48494C1F388068AB
:100CA000A178884200D2A0704949A2785F39822099
:100CB00001F067FD032060704548A2788168891AB9
:100CC00081600021017310BD414810B51F38816853
:100CD00039B1007B000601D5822000E0022001F03E
:100CE0000BFD3B4900200873BDE81040D0E610B56D
:100CF000FFF7BDFF00281FD0354870215F38022262
:100D00000170002141708270C17001714171817167
:100D10000A22C271017241728172C1723022027361
:100D2000012242738173C1730174417424491220FA
:100D30008870BDE81040AEE710BD1CB5FFF797FF07
:100D400000286AD02A480A2206210388684600F053
:100D500025FA1F4800225F3880230270437082709A
:100D60000121C1702021017143718271C271412240
:100D70000272542242724F2282724C22C27201735A
:100D800041738173C17346220274502343747223EA
:100D900083746923C3746E2303757423437581754B
:100DA000C2756C22027661224276732282766822B4
:100DB000C276017741778177C1779DF8011019E0FC
:100DC00078000010E051000039020010B11C001042
:100DD000981C00105553425300C0092000000940E0
:100DE000A0860100BC00001020A1070068000010D0
:100DF0000404000080F820109DF8021080F82110F3
:100E00009DF8031080F822109DF8041080F823103C
:100E1000DE4924208870FFF73EFF1CBD10B5FFF7A8
:100E200026FF00280CD0DA48032101700021417010
:100E30008170C170D54904208870BDE810402AE750
:100E400010BD10B5FFF713FF002810D0D0480021C7
:100E50000622017042708170C1700171417181710F
:100E6000C171CA4908208870BDE8104013E710BD61
:100E700010B5FFF7FCFE002815D0C44AC448116A1B
:100E8000491E0B0E03700B0C43700B0A8370C1706C
:100E900000210171417102238371C171082090709A
:100EA000BDE81040F7E610BD10B5FFF7E0FE0028E2
:100EB00019D0B7480021B54B0170417081700822EC
:100EC000C2701A6A140E0471140C4471140A8471ED
:100ED000C2710222027241728272C1720C20987039
:100EE000BDE81040D7E610BD2DE9F041A74DA84C54
:100EF0000021A8784034A64A02E0535C6354491CA0
:100F000003468142F9D31F2B72D12068A149884240
:100F10006ED19F4E60685F364FF001087060A06828
:100F2000B060607B18B9A07B08B1102802D986F8A0
:100F30000C8059E0E07B1E28F9D00FDC12282ED05F
:100F400005DC48B30328F2D1BDE8F041CFE615280F
:100F5000EDD01A28EBD1BDE8F0415FE702272A283F
:100F600028D010DC23281DD025281ED02828DED12B
:100F7000FFF75AFE002826D0207B000618D56F7098
:100F8000BDE8F04159E52F281ED05528CFD05A286A
:100F9000CDD1BDE8F04154E7BDE8F04194E6BDE8AD
:100FA000F041CAE6BDE8F0417EE7BDE8F0415FE709
:100FB000022016E0FFF738FE002804D0207B000650
:100FC0000ED485F801802DE6FFF72EFE0028FAD01A
:100FD000207B000604D485F80180C5F8288021E62E
:100FE000822001F089FB3773BDE8F04150E5FFE74F
:100FF000822001F081FB022001F07EFB0620687058
:1010000010E6624810B54178022908D003290ED0B5
:1010100004290FD0052901D10021417010BD5C4881
:101020004030C07B2828F9D1BDE8104005E5BDE877
:1010300010402DE5822001F05FFBF8E710B5544920
:10104000022001F06DFB51498870487858B10128A1
:101050000CD0022001F050FB4D4902205F31087393
:10106000BDE8104014E5BDE810403DE74848403079
:10107000C07B2A2804D02F2805D1BDE8104098E570
:10108000BDE810406CE510BDFFB50246002002EB44
:10109000420501464FF440566C4603AA6B1844F8CB
:1010A0002130B34202DD002004B0F0BD3A4F07EB1F
:1010B0006307DB073F78575401D03B095354535C17
:1010C0008F0003F00F035354BB40491C18440329FD
:1010D000E4DBE9E7F0B506460020034602462E4C65
:1010E0004FF4007700E05B1CF55C45B102EB030CAC
:1010F000A4440CF5805C9CF800C8AC45F3D0032BED
:101100003FD302F5C0502044037F457FC67F03EBE9
:101110000523857F2D0405EB06652B4451EA030565
:101120002BD021B91949496840318B4225D8184B39
:1011300000216C335518254405F5805595F8005865
:101140005D54491C0C29F5D3817EC27E01EB02213E
:10115000027D407D120402EB00600C182046FFF770
:1011600093FF40F6F57501E0FFF78EFFC11EA9421F
:10117000FAD3A0F57061FF3901D00020F0BD204600
:10118000F0BD2032BA42AFD3F0BD000078000010AD
:10119000391C00105553424339020010FFB5B1A667
:1011A0000446E1CE8DE8E100022902DA002004B015
:1011B000F0BD6018002100F8011D6946B3FBF2F58F
:1011C00002FB1535B3FBF2F34D5D00F8015DA04263
:1011D000F4D8ECE710B503F02AFC03F014FCA549A1
:1011E0004FF40052C1E90020A0F5F420886010BD42
:1011F00070B5034608468D189E49002449688D4203
:1012000000D9881A194603F061FC204670BDF8B574
:101210001446984E0A460B19716800258B4200D976
:101220000A1B03460094306803F07BFC2846F8BD97
:1012300010B50B4601460024184603F01BFC20465F
:1012400010BD2DE9FC410746002090460E46ADF842
:10125000000004460EE0351B402D00D94025391909
:101260002A468548FFF7E4FFAAB283496846FEF79D
:1012700083FF2C44B442EED33919424601A8FFF74C
:10128000D7FFBDF80000BDF80410884202D101204C
:10129000BDE8FC810020FBE70021425C12B9491C3B
:1012A0001829FAD3182901D000207047012070476F
:1012B0002DE9F0436F4C00200C348BB0A070E0702F
:1012C000DFF8B8816E4F4FF4005620714FF48079EB
:1012D0000125192231466846FFF7AAFF022216218E
:1012E0003046FFF7AEFF00287ED0DDF80E10022258
:1012F00006F11900FFF7A5FF002875D09DF8001032
:10130000062929D2DFE801F029030329291CD8F88E
:101310007420DDF80A30521C93421DD2D8F87400B4
:10132000DDF80A30C01ADDF80E30401C984213D3A5
:10133000DDF80A00DDF80E30184490420CD80CE0BD
:10134000DDF80E00B0F5F42F00D9A570DDF812001D
:10135000C0F30B40152800D0A570012903D0022945
:1013600001D0052943D19DF808004A46400706F2FE
:10137000194107D54348FFF75BFF41494148FEF754
:101380000EFF02E03E48FFF753FF00200990B888A7
:10139000ADF824000999019889B2884200D0A5705F
:1013A00000200990387B8DF824000999BDF80100D0
:1013B000C9B2884200D0A5709DF80000022816D15D
:1013C000386B0990DDF812000999884200D0A570A9
:1013D0000020099097F834008DF8240009999DF8B1
:1013E0000300C9B2884200E025E000D0A5709DF856
:1013F0001800401EFE2800D2A570BDF80100A0F51F
:101400007F41FF3901D04E2802D19DF8030020B959
:101410006846FFF741FF00B9A570DDF80E001B36E6
:1014200006446846FFF738FF30B1E07880B1217993
:1014300088420DD012E0A5709DF8180010B92079EF
:10144000401C2071E078401CC0B2E0700C2801D331
:10145000A57003E0A07800283FF43BAFA0780BB064
:10146000BDE8F083303132333435363738394142D4
:1014700043444546B0000010B11C001098520000D3
:10148000B11E0010B11D00104F4A104710B572B6C2
:1014900033244E4B10C307C34D484FF47A71006894
:1014A000B0FBF1F01860191D4848FFF7EDFF62B678
:1014B00010BD464A32231360C2E9010144484FF48B
:1014C0007A710068B0FBF1F0D06002F114011046AF
:1014D000DAE73E4A34231360C2E901013C484FF485
:1014E0007A710068B0FBF1F0D06002F1140110468F
:1014F000CAE710B572B60624364900BF51F8242059
:10150000824212D93349783951F82410814207D1E7
:1015100021460846FFF7CDFF21460846FFF7D9FFD1
:1015200021460846FFF7C5FF02E0641C1D2CE5D9E3
:1015300062B610BD2DE9F041274C236803B9206045
:10154000224D00202835636803E00F5C1E18401C04
:10155000AF559042F9D398184FF480766060B0424E
:1015600013D12068FFF7C5FF184D1435286800B166
:10157000FEE71649324628312068FFF787FF2868C2
:1015800000B1FEE70020606020600020BDE8F0812F
:1015900072B61249124A01401160FEF7E9BD46F2E7
:1015A000044000210088A0F51942993A0AD04FF46E
:1015B000C0404FF4002208C890421944FBD309B13F
:1015C0000020704701207047F11FFF1FB41F00105B
:1015D000D800001098520000C400001080FFFF1FC8
:1015E00008ED00E0002070477A49820702D54FF4E9
:1015F00000128A61C20702D04FF480728A614207EA
:1016000002D54FF400228A61000702D54FF4801002
:101610008861002070476F49820702D54FF400129D
:10162000CA61C20702D04FF48072CA61420702D574
:101630004FF40022CA61000702D54FF48010C86140
:101640000020704701460020624A8B0703D553698A
:101650009B0200D50220CB0704D05369DB0501D5DE
:1016600040F001004B0704D553691B0301D540F03E
:101670000400090704D55169C90201D540F00800EA
:10168000704710B50446FFF7DDFF0346FFF7C3FFC1
:1016900024EA0300FFF7A8FF002010BD70B54E4BF1
:1016A00050B15968042403250226052907D2DFE832
:1016B00001F0072B4A708D0000205860986070BDC3
:1016C000042807D0052809D00124022879D0012850
:1016D00008D00FE00F20FFF79EFF45E0BDE8704007
:1016E000012098E70F20FFF796FF0BE0FFF77CFF44
:1016F0005C6070BD0E28FCD10F20FFF78CFF02202C
:10170000FFF772FF0120F1E706280AD0032810D066
:101710000A2813D0092811D00D280FD00C28D9D0B1
:1017200070BD0F20FFF777FF0220FFF75DFF5E60BF
:1017300070BD0F20FFF76FFF012026E00F20FFF79D
:101740006AFF022011E0062812D00A2819D00928C1
:10175000C8D00C28BED00D28F0D00F28E8D1FFF754
:101760005AFF0220FFF740FF0120BDE870403BE731
:10177000986810F01F0F00F101009860D8D1022086
:101780001BE00F20FFF747FF0220FFF72DFF5D60F2
:1017900070BD072806D00A289CD00B2811D0092834
:1017A000A0D070BD0220FFF736FF986810F03F0F01
:1017B00000F101009860F4D10120BDE8704060E7BD
:1017C000FFE70F20FFF727FF02208FE70628A8D0AA
:1017D00090E7000000C00920CC0000104F4810B571
:1017E0002021C0F8A01100BFD0F8A0114906FBD5F8
:1017F0000521C0F804114FF04472C0F8A8214FF43D
:101800008062C0F8AC210122C0F80C210B23C0F883
:101810008430C0F88020AA22C0F88C205523C0F85C
:101820008C3000BFD0F888406401FBD50324C0F899
:101830008040C0F88C20C0F88C30C0F808113849BE
:10184000C0F8C4100021C0F8C811D0F888106FEAA1
:1018500011618A073349D0F80C2102F0030207D046
:101860007AB3012A44D0022A47D0032A4ED13AE063
:101870002AB1012A13D0022A24D0032A46D1D0F853
:101880008820D0F80431C2F30742DBB2521C5B1C43
:101890005A43D0F88830244CC3F30E030EE0D0F83E
:1018A0008820D0F80431C2F30742DBB2521C5B1C23
:1018B0005A43D0F888301D4CC3F30E035B1C6343BE
:1018C00021E010E0D0F88820D0F80431C2F30742BC
:1018D000DBB2521C5B1C5A43D0F888304FF47A4478
:1018E000C3F30E03EAE7D0F80421114BD2B209E0AA
:1018F000D0F804210F4BD2B204E0D0F804214FF409
:10190000FA43D2B2521CB3FBF2F20A60016821F42E
:10191000704141F40051016010BD000000C00F4053
:10192000DE96E883D800001000127A0000366E01BF
:1019300000093D00001BB700434900200867C8604C
:1019400010224A618861C022CA6340498A684049BE
:10195000C1E900203F4908603F49086078463F4997
:101960000860002070472DE9F04341F288320023DF
:10197000384C394D394E904208D8642800D228B9E5
:1019800042F21072914201D8052907D286202060C8
:1019900078462B6030608620BDE8F083DFF8AC909D
:1019A000D9F80820DFF8A880D8F80070D21BD8F842
:1019B000047007EB470CCCEBC717B2EBC70F06D28E
:1019C0000520206078462B6030600520E4E71E4A41
:1019D00002275760D2F83CC00CF0FD0CC2F83CC0A6
:1019E00040B1DFF87CC0BCFBF0F04010D061576024
:1019F00001205060D9F80800C8E90001236078464A
:101A00002B6030600020C7E770B5114C00250E46F2
:101A10006560FFF7A8FF0F49000601D5086870BD93
:101A20000A4B06EB46022068C2EBC6129E68361AC5
:101A3000B6EBC20FFAD3044802224260C26B02F036
:101A4000FD02C2636560E9E70080004000000940D4
:101A5000E00000106C000010700000107400001016
:101A6000001BB70030B5FF4800218162016921F4F5
:101A700040710161016D21F4407141F40071016513
:101A8000F9491022CA650B6C43F010030B6483689C
:101A900023F440738360836C23F4407343F4007336
:101AA0008364CA630B6A23F010030B62836823F01C
:101AB00003038360836C23F003039B1C8364012472
:101AC0008C630B6A43F001030B62836823F00C0301
:101AD0008360836C23F00C0343F0080383640223C8
:101AE000CB630B6A43F002030B62436A23F040733B
:101AF00043F000734362436E23F0407343F000737E
:101B00004366436A23F0406343F000634362436EDD
:101B100023F0406343F000634366C36823F04073DF
:101B2000C360C36C23F0407343F00073C3641306B7
:101B3000CB630B6A43F080530B62036923F4405379
:101B40000361036D23F4405343F4005303654023C2
:101B50008B650D6C45F040050D64056925F00305A6
:101B60000561056D45F0030505658C650C6C44F059
:101B700001040C64046824F4404444F40044046008
:101B8000046C24F440440464046824F4402444F4C1
:101B900000240460046C24F440240464446824F0A9
:101BA00030044460446C24F0300444F02004446465
:101BB0009403CC610D6825F480250D60C56845F05F
:101BC0004045C560C56C25F0404545F00045C564FD
:101BD000056825F0300545F010050560056C25F019
:101BE000300545F020050564056825F0C00545F081
:101BF00040050560056C25F0C0050564056825F005
:101C0000404545F080450560056C25F0404545F0B0
:101C100000450564456825F003056D1C4560456C6D
:101C200025F003054564056925F4403545F4003584
:101C30000561056D25F4403545F4003505650569F8
:101C400025F4402545F400250561056D25F4402562
:101C50000565056825F00305AD1C0560056C25F0DC
:101C60000305AD1C0564056825F00C0545F0080565
:101C70000560056C25F00C050564C56845F4403524
:101C8000C560C56C25F4403545F40035C564C568AC
:101C900045F44045C560C56C25F4404545F4004514
:101CA000C564C56845F44075C560C56C25F44075CC
:101CB00045F40075C564C56825F44055C560C56C1C
:101CC00025F44055C56495048D630D6A45F480057F
:101CD0000D62C56825F03005C560C56C25F030057E
:101CE000C5648C630C6A44F480240C62446824F05C
:101CF000407444F080744460446C24F04074446444
:101D0000446824F4400444F480044460446C24F4A3
:101D100040044464446824F0406444F080644460B7
:101D2000446C24F0406444F000644464446824F04B
:101D3000405444F080544460446C24F0405444F0D7
:101D400000544464C46824F0405444F00054C46017
:101D5000C46C44F04054C464C46924F44024C46195
:101D6000C46D44F44024C4655405CC670C6E44F043
:101D700000740C66446824F4404444F48044446095
:101D8000446C24F4404444F400444464446824F41F
:101D9000403444F480344460446C24F4403444F4CB
:101DA00000344464446824F4402444F480244460AF
:101DB000446C24F4402444F400244464446824F42F
:101DC000401444F480144460446C24F4401444F4FB
:101DD00000144464C46844F44024C460C46C24F413
:101DE000402444F40024C464C46824F00304C460A0
:101DF000C46C24F00304A41CC46414038C630C6A34
:101E000044F480340C62046924F440040461046DD9
:101E100024F440040465C414CC650D6C25F40065FD
:101E20000D64056825F440350560056C25F44035E2
:101E300045F4003505648515CD610D6845F4807560
:101E40000D60456825F440654560456C25F44065A6
:101E500045F4006545645504CD610D6845F40015F1
:101E60000D6003E000C0024000C00920456825F471
:101E700040754560456C25F4407545F40075456432
:101E80001504CD610D6845F480150D60456825F099
:101E9000C0054560456C25F0C00545F080054564EA
:101EA000D503CD610D6845F400250D60C56825F4A6
:101EB000400545F48005C560C56C25F4400545F432
:101EC0000005C564056825F440550560056C25F4DA
:101ED00040550564CB610B6823F040030B60C36978
:101EE00023F44013C361C36D23F4401343F4001380
:101EF000C3659305CB670B6E43F080630B66036885
:101F000023F440730360036C23F440730364CA61D9
:101F10000A6822F010020A60026822F4406202603D
:101F2000026C22F4406202642022CA610B6823F032
:101F300020030B60836823F440138360836C23F4D5
:101F4000401343F4001383640315CB630D6A45F417
:101F500080650D62856825F040558560856C25F0AB
:101F6000405545F0005585645502CD630D6A45F432
:101F700080450D62056825F440050560056C45F453
:101F800040050564CC610C6824F400640C600468AE
:101F900024F440140460046C44F440140464CB61E1
:101FA0000B6823F480630B60036923F440630361CF
:101FB000036D43F440630365CA65086C40F020007C
:101FC000086430BDFA4800214FF001128180017091
:101FD0004170C0E902217047F5491C31002000F032
:101FE0009FBB10B5F24C1434A288402A00D940227D
:101FF0008020216800F0C5FB216801442160A18890
:10200000081AA08010BD10B5E94C002014342168D6
:1020100000F086FB216801442160A188081AA08095
:1020200010BD00221146802000F0ABBBE14900202A
:1020300000F076BB70B5DE48DD4D1C3005F11405AF
:10204000007810F01F040AD0D949DA4B01F11C00C6
:102050004A780079012C06D0022C26D109E0D44818
:10206000001D28601DE002B3897888421DD200203F
:1020700015E000F08F04200605D504F00F064FF49C
:102080008030B04001E00120A0400AB922070CD105
:102090008A68024209D0C9680142E8D0012018804C
:1020A0002B60FFF79EFF012070BD002070BD02462F
:1020B00070B5BF48BE4C1C30017811F01F030146BB
:1020C000498804D0012B29D0022B27D111E0012906
:1020D00024D132B1012000F0BDFAA08840F0020006
:1020E00005E0002000F0B6FAA08820F00200A080F1
:1020F00021E0007900F08F00030605D500F00F0302
:102100004FF480359D4001E00125854063782BB177
:10211000030703D0A3682B4200D009B1002070BD93
:1021200022B100F0E9FAE068284303E000F0EEFA9B
:10213000E068A843E060012070BD9D4810B51C30E8
:10214000007810F01F0F9A4800F11C00C0782AD1C7
:1021500097491431012807D001F108020228937829
:1021600006D003281FD112E093480860122012E025
:102170009248002204E004780CB144882044521CA8
:102180009342F8D1027872B10860408803E08C482D
:102190001844086000788A88824200D98880FFF756
:1021A00020FF012010BD002010BD2DE9F84F804F09
:1021B00000201C370090B8787D4E4FF000094FF09A
:1021C000010A4FF4803B00286BD07C4C65E06078BE
:1021D000022804D0042841D005285CD141E061796F
:1021E000B878814238D170702079B0707049002081
:1021F00011F1100101F80090401C0428FAD30125C8
:102200004FEA06080AFA05F0D8F80810084202D08A
:10221000284600F05DFAD8F808100BFA05F00842DD
:1022200003D045F0800000F053FA6D1C102DE9D367
:102230004FF00110C8E90209012000F00CFAE07922
:102240004006B8F8040002D540F0010001E020F09B
:102250000100A8F804001EE060881DE0E07800900E
:1022600019E00098B8B9A07800F08F05280604D5C9
:1022700005F00F010BFA01F001E00AFA05F0B16870
:1022800001432046B16000F0FCF9284600F016FA40
:10229000284600F027FA207804442078002896D1B8
:1022A0001FE086F8019001245546D846B16805FA2A
:1022B00004F0084202D0204600F00AFAB16808FA99
:1022C00004F0084203D044F0800000F001FA641CDE
:1022D000102CEBD34FF00110C6E90209002000F0EA
:1022E000BAF9B8787178884202D10120BDE8F88F38
:1022F0000020FBE72DE9FC5F2D4D00273E46687866
:10230000BB46B846002871D0BA462C4C05F11C09D2
:1023100068E06078022804D0042808D005285FD13E
:1023200019E06079697888425AD0608859E0A778C6
:1023300099F80410E6784FF00008B94250D199F8A6
:102340000200B0424CD11A484FF0010A103010F888
:1023500007B0C65544E099F80410B94240D1A178BD
:1023600001F08F010191090605D5019901F00F02D5
:102370004FF4803101E0019A01219140009199F8D8
:102380000200B0421ED1A8680843A860E96800981E
:1023900081432046E96000F074F9019800F08EF95D
:1023A000019800F09FF9009948EA010818E0000040
:1023B000E8000010DC200010105300002253000041
:1023C000435300005E450BD118EA010F08D1A868FD
:1023D0008843A860E8688843E860019800F078F9CD
:1023E000207804442078002893D15046BDE8FC9F13
:1023F0002DE9F041494C0027A4F108062178A4F109
:102400001C05082863D2DFE800F06204647262628F
:102410008381FFF7E1FD2078C00900F04EF9E088E4
:10242000B0802078C0F34111F1BB61780C294AD209
:10243000DFE801F00609490B49101A1D1F2531423A
:10244000FFF7F8FD4DE0002000E00120FFF72FFE30
:1024500050B306E010F01F0F35D1A07840F0800097
:102460002870BDE8F041DCE5FFF767FE39E00020A9
:102470002AE010F01F0F26D128481B381AE010F070
:102480001F0F20D1FFF791FE70B1FFF7CAFDBDE825
:10249000F041FDF77DBF00F01F00012813D16878DF
:1024A00010B12079A97800E00DE088420BD21B49D9
:1024B0000C39084430601CE000F01F00012802D1F4
:1024C000FFF718FFC4E7802000F016F9B780BDE8D9
:1024D000F081080608D4B0880028F8D0FFF793FDF3
:1024E000B0880028EFD0F2E7BDE8F0419EE508068D
:1024F00002D5BDE8F04174E528780106E7D500F083
:102500007F002870BDE8F04100F054B8802000E062
:102510000020BDE8F04100F0F9B80000040100100F
:1025200001460007C00E090600D5401C7047DA4975
:102530001022C1F80822C1F8100200BFD1F8000231
:10254000C006FBD57047D44A1023C2F80832C2F83F
:10255000100200BFD2F80002C006FBD5C2F8083254
:10256000C2F81012D2F80002C006FBD57047CA4963
:102570003022C1F80822C1F8100200BFD1F80002D1
:102580008006FBD5D1F81402704710B5040001D0C5
:10259000012000E000204FF4807141EA0041BF4873
:1025A000FFF7D1FFBE494FF000700CB1886710BD36
:1025B000C86710BD30B5BB49BB4D41EA0044214658
:1025C0002846FFF7C0FF21462846BDE83040BAE75D
:1025D000B1480021C0F848124021C0F84C12012235
:1025E000C0F84822C0F84C12D0F80012C905FBD53B
:1025F0004FF0FF31C0F83812C0F83412C0F808129A
:102600000C21C0F804127047A84800B5C16821F039
:10261000405141F00051C160C16C41F04051C16472
:10262000A3491A200860091D0A6830EA0202FBD19A
:102630004FF0E0214FF08070C1F880029D4B2022C6
:1026400083F80024C1F80001FFF7C2FF00205DF805
:1026500004EBAFE7704710B500B101204FF4807470
:1026600044EA00419448FFF76EFF8B480321C0F80D
:10267000441200BFD0F80012C905FBD5C0F80842CB
:1026800010BD10B502468078FFF74AFF8249D1F8A5
:102690004432012484402343C1F84432C1F8480243
:1026A0009088C1F84C0200BFD1F80002C005FBD5EC
:1026B0004FF48070C1F8080210BD704700B5FFF7F5
:1026C0002FFF7E495DF804EB41EA004089133AE7A9
:1026D00000B5FFF725FF79495DF804EB41EA0040BA
:1026E000774930E700B5FFF71BFF74495DF804EB4D
:1026F00041EA0040891326E700B5FFF711FF6F4953
:102700005DF804EB41EA00406E491CE700B5FFF7B5
:1027100007FF6A495DF804EB41EA0040891312E7BC
:1027200000F00F02012370B503EB82035A4AC2F88E
:10273000283200BFD2F820321C05FBD5C3F30903B1
:102740000024DD1C05E000BFD2F8186241F8046BDC
:10275000641CB4EB950FF7D30021C2F8281241F2A4
:102760004821C140C9070AD1FFF7DAFE4FF4A06142
:1027700041EA0040FFF7DBFE5348FFF7D8FE18465A
:1027800070BD70B513460546434C00F00F000222A1
:1027900002EB8000C4F82802C4F824320020DA1CBE
:1027A00005E000BF51F8046BC4F81C62401CB0EB9C
:1027B000920FF7D30020C4F828022846FFF7B0FE96
:1027C0004FF4A06141EA0040FFF7B1FE3F48FFF738
:1027D000AEFE184670BD2DE9F0412F4DD5F8003200
:1027E000C5F80832180721D52C48FFF7A0FE384855
:1027F000FFF7BDFEC10605D5FFF7EAFEBDE8F041D3
:10280000FDF7B7BD810705D5BDE8F04100F0010037
:10281000FDF7A9BD010709D5400703D5BDE8F04183
:10282000FDF7AEBDBDE8F041FDF7B1BD294E58073B
:102830004FF001071CD4BDE8F0810024D5F8302208
:1028400007FA04F10A4210D06008C5F8381200BF38
:10285000D5F800128906FBD5D5F81412E2070CD082
:1028600056F8201009B103208847641C202CE5D3BA
:10287000D5F830020028E0D1DDE73CB9490705D59D
:10288000316819B1012088470124D7E756F8201094
:102890000029EAD00220E7E700C000500005FE0052
:1028A00000C00920000180000005D00000C00240E7
:1028B000F4CF005018E000E00005D800000540000B
:1028C00000012000000101000005F2000005FA00EF
:1028D0000002FE00B45300002DE9F047F74E804699
:1028E0004FF080773068BC11F54DB84249D100BF38
:1028F00000BF00BF00BF00BF00BF00BF00BF00BFE0
:1029000000BF00BF00BF00BF00BF00BF00BF00BFCF
:1029100000BF00BF00BF00BF00BF00BF00BF00BFBF
:1029200000BF00BF00BF00BF00BF00BF00BFEC631F
:102930001520FDF7A9FC0020FDF7A6FC00F0FF091B
:10294000AC6300BF00BF00BF00BF00BF00BF00BF3F
:1029500000BF00BF00BF00BF00BF00BF00BF00BF7F
:1029600000BF00BF00BF00BF00BF00BF00BF00BF6F
:1029700000BF00BF00BF00BF00BF00BF00BF00BF5F
:1029800000BF00BF00BF00BF00BF00BF00BF00BF4F
:1029900000BF00BF00BF00BF00BF00BF00BF00BF3F
:1029A00000BF00BF00BF00BF00BF00BF00BF00BF2F
:1029B00000BF00BF00BF00BF00BF00BF00BF00BF1F
:1029C00000BFEC630620FDF75FFCAC6300BF00BFF7
:1029D00000BF00BF00BF00BF00BF00BF00BF00BFFF
:1029E00000BF00BF00BF00BF00BF00BF00BF00BFEF
:1029F00000BF00BF00BF00BF00BF00BF00BF00BFDF
:102A000000BF00BF00BF00BF00BF00BF00BF00BFCE
:102A100000BF00BF00BF00BF00BF00BF00BF00BFBE
:102A200000BF00BF00BF00BF00BF00BF00BF00BFAE
:102A300000BF00BF00BF00BF00BF00BF00BF00BF9E
:102A400000BF00BF00BF00BF00BF00BFEC6301209C
:102A5000FDF71AFC4FEA8800FDF716FC3068B84213
:102A600002D14846FDF710FCAC6300BF00BF00BFB9
:102A700000BF00BF00BF00BF00BF00BF00BF00BF5E
:102A800000BF00BF00BF00BF00BF00BF00BF00BF4E
:102A900000BF00BF00BF00BF00BF00BF00BF00BF3E
:102AA00000BF00BF00BF00BF00BFBDE8F0872DE939
:102AB000FC5F8846044601A9824800F05DFB824D18
:102AC000824E834FF0BB03208DF8000020098DF863
:102AD000010020018DF802004FF000098DF80390ED
:102AE00000BF00BF00BF00BF00BF00BF00BF00BFEE
:102AF00000BF00BF00BF00BF00BF00BF00BF00BFDE
:102B000000BF00BF00BF00BF00BF00BF00BF00BFCD
:102B100000BF00BF00BF00BF00BF00BF00BF00BFBD
:102B2000DFF89CB14FF4802ACBF83CA00421684622
:102B3000FDF7B1FB00240020FDF7A6FBC0B28DF825
:102B4000040000E003E018F80410884208D0822056
:102B5000286022203060784638608220BDE8FC9FE3
:102B6000641CB4F5805FE6D3CBF838A000BF00BF8B
:102B700000BF00BF00BF00BF00BF00BF00BF00BF5D
:102B800000BF00BF00BF00BF00BF00BF00BF00BF4D
:102B900000BF00BF00BF00BF00BF00BF00BF00BF3D
:102BA00000BF00BF00BF00BF00BF00BFC5F800905E
:102BB0007846C6F8009038600020CFE72DE9F0474E
:102BC0004FF0000900BF00BF00BF00BF00BF00BF43
:102BD00000BF00BF00BF00BF00BF00BF00BF00BFFD
:102BE00000BF00BF00BF00BF00BF00BF00BF00BFED
:102BF00000BF00BF00BF00BF00BF00BF00BF00BFDD
:102C000000BF00BF2E4E4FF48025F5639F20FDF7D7
:102C10003BFB0020FDF738FB00F0FF080020FDF72C
:102C200033FBC4B20020FDF72FFBC1B2B56300BF78
:102C300000BF00BF00BF00BF00BF00BF00BF00BF9C
:102C400000BF00BF00BF00BF00BF00BF00BF00BF8C
:102C500000BF00BF00BF00BF00BF00BF00BF00BF7C
:102C600000BF00BF00BF00BF00BF00BF00BF164DC8
:102C7000164E174FB8F1C20F01D1202C07D0822079
:102C80002860212030607846386082200DE70B48AC
:102C900014291FD0152920D0162922D0182923D075
:102CA000C0F800900020FFF717FEC5F800907846A6
:102CB000C6F8009038600020F7E60000140100100C
:102CC00000C00920A08601006C00001070000010F8
:102CD000740000104FF4801101E04FF40011016006
:102CE000E0E74FF48001FAE74FF08071F7E72DE954
:102CF000F34FC3B0804600244FF0820AFE4DFF4ED2
:102D0000FF4F4FF0210BA14641A9FE4800F034FAD5
:102D100000286CD100F09CFA02208DF800004FEAE8
:102D200018108DF8010004EB08108DF8020044988B
:102D30008DF8039000EB04214FF4807201A801F09C
:102D40008BFF00BF00BF00BF00BF00BF00BF00BFC0
:102D500000BF00BF00BF00BF00BF00BF00BF00BF7B
:102D600000BF00BF00BF00BF00BF00BF00BF00BF6B
:102D700000BF00BF00BF00BF00BF00BF00BF00BF5B
:102D800000BFE1494FF48020C8634FF48271684668
:102D9000FDF781FADC494FF48020886300BF00BF53
:102DA00000BF00BF00BF00BF00BF00BF00BF00BF2B
:102DB00000BF00BF00BF00BF00BF00BF00BF00BF1B
:102DC00000BF00BF00BF00BF00BF00BF00BF00BF0B
:102DD00000BF00BF00BF00BF00BF00BF641CE4B263
:102DE000102C91D341A9C74800F0C6F948B1C5F8E5
:102DF00000A07846C6F800B03860822045B0BDE833
:102E0000F08F00F06FFAC5F800907846C6F8009091
:102E100038600020F2E72DE9F04F89B0DFF8D88262
:102E20005FEA020B4FF0000607910FD04FF4805578
:102E300001462A466846FDF749FADDE9004728467B
:102E400001F0B4FE5FEA00090CD016E08621AB4821
:102E5000C8F80010092101607946A9480160862060
:102E600009B0CCE78221A548C8F8001022210160F2
:102E70007946A34801608220F2E7ABEB0605C7F56F
:102E800080504FF0000AA84200D20546B5F5805F99
:102E900004D02046494600F0A3FCD8B907982A463A
:102EA000811907EB090001F0D7FE204600F01DFC58
:102EB00080B920464946FFF71AFF58B920464946CF
:102EC000FFF7F5FD78B10AF1010000F0FF0ABAF151
:102ED000030F05D3484601F098FED8F80000BFE77D
:102EE000BAF1000FE1D12E440027641C5E45C4D323
:102EF000484601F08AFE81490020C8F800000860B9
:102F000079467F4801600020AAE72DE9FF4F8DB088
:102F10000D46DDF868900026774C07935FEA0901BB
:102F20003FD04FF4805701463A466846FDF7CEF948
:102F3000DDE900B10C913A46691C6846FDF7C6F917
:102F4000DDE90010CDE904013A4668460F99FDF726
:102F5000BDF9DDE9008500BFA9EB0607C5F5805086
:102F6000B84200D2074625B1D8457CD10C9885429D
:102F700079D14FF4805001F019FE5FEA000A1BD0AE
:102F8000D8454FD10C9885424CD12A464FEA08309B
:102F9000514600F0FEFA000618D5504601F035FE05
:102FA00079E086202060554809210160784654491F
:102FB0000860862011B022E7822020604F4822213D
:102FC000016079464E4801608220F3E7059880450C
:102FD00009D1049901EB0030C1F58052514400F051
:102FE000D8FA0006D9D4404600F07FFB0006D4D4BE
:102FF00007983A46811905EB0A0001F02DFEEA19FF
:103000004FEA0830514601F0DCF90006C5D40599B5
:10301000884533D1049800EB01300499C1F5805202
:10302000514427E0059988450AD1049800EB013006
:103030000499C1F58052514600F0ABFA0006ACD4B9
:10304000404600F052FB0006A7D407983A46811983
:103050000F98304401F0B5F900069ED405998845D3
:103060000CD1049800E00DE000EB01300499C1F5AB
:103070008052514601F0A5F900068ED4504601F069
:10308000C4FD0AE007983A4681190F98304401F0D0
:1030900098F9000601D520688CE73E44002508F128
:1030A00001084E45FFF458AF144900202060086025
:1030B00078461349086000207CE714480068704790
:1030C0004FF4805070472DE9F04FDFF82C80DFF887
:1030D0002CB089B00F0004464FF0000633D04FF4F7
:1030E000805501462A466846FDF7F0F8DDE900A163
:1030F00005912A4621460BE06C000010700000107C
:1031000074000010A086010000C009201401001006
:1031100006A8FDF7DBF8DDE906404FF00009BD1B0E
:10312000C0F58051A94200D20D4620B1544515D1B9
:103130000599884212D1204600F0D7FA00060DD535
:10314000D8F800008CE68621C8F800100921CBF8D9
:10315000001079463B480160862081E62E44641CBD
:103160004846BE42DBD3C8F800007946CBF80000E1
:1031700034480160002073E62DE9F041324C0F46DF
:103180000646A56806E0A068401BB04202D30120B5
:10319000BDE8F081384600F003F80028F3D1F7E7E6
:1031A00070B5044600BF00BF00BF00BF00BF00BF36
:1031B00000BF00BF00BF00BF00BF00BF00BF00BF17
:1031C00000BF00BF00BF00BF00BF00BF00BF00BF07
:1031D00000BF00BF00BF00BF00BF00BF00BF00BFF7
:1031E00000BF00BF194E4FF48025F5630520FDF7A1
:1031F0004BF80020FDF748F82070B56300BF00BF12
:1032000000BF00BF00BF00BF00BF00BF00BF00BFC6
:1032100000BF00BF00BF00BF00BF00BF00BF00BFB6
:1032200000BF00BF00BF00BF00BF00BF00BF00BFA6
:1032300000BF00BF00BF00BF00BF00BF207800F08C
:10324000010070BD740000100000094000C009209A
:1032500070B500BF00BF00BF00BF00BF00BF00BF10
:1032600000BF00BF00BF00BF00BF00BF00BF00BF66
:1032700000BF00BF00BF00BF00BF00BF00BF00BF56
:1032800000BF00BF00BF00BF00BF00BF00BF00BF46
:1032900000BFFE4C4FF48025E5630620FCF7F4FFE9
:1032A000A56300BF00BF00BF00BF00BF00BF00BFDD
:1032B00000BF00BF00BF00BF00BF00BF00BF00BF16
:1032C00000BF00BF00BF00BF00BF00BF00BF00BF06
:1032D00000BF00BF00BF00BF00BF00BF00BF00BFF6
:1032E00000BF70BD70B500BF00BF00BF00BF00BF12
:1032F00000BF00BF00BF00BF00BF00BF00BF00BFD6
:1033000000BF00BF00BF00BF00BF00BF00BF00BFC5
:1033100000BF00BF00BF00BF00BF00BF00BF00BFB5
:1033200000BF00BF00BFD94C4FF48025E5630420E7
:10333000FCF7AAFFA56300BF00BF00BF00BF00BF2E
:1033400000BF00BF00BF00BF00BF00BF00BF00BF85
:1033500000BF00BF00BF00BF00BF00BF00BF00BF75
:1033600000BF00BF00BF00BF00BF00BF00BF00BF65
:1033700000BF00BF00BF70BD70B5064600BF00BFF4
:1033800000BF00BF00BF00BF00BF00BF00BF00BF45
:1033900000BF00BF00BF00BF00BF00BF00BF00BF35
:1033A00000BF00BF00BF00BF00BF00BF00BF00BF25
:1033B00000BF00BF00BF00BF00BF00BFB34D4FF450
:1033C0008024EC635020FCF75FFFAC6300BF00BFBC
:1033D00000BF00BF00BF00BF00BF00BF00BF00BFF5
:1033E00000BF00BF00BF00BF00BF00BF00BF00BFE5
:1033F00000BF00BF00BF00BF00BF00BF00BF00BFD5
:1034000000BF00BF00BF00BF00BF00BF00BF00BFC4
:1034100000BF00BF00BF00BF00BF00BF00BF00BFB4
:1034200000BF00BF00BF00BF00BF00BF00BF00BFA4
:1034300000BF00BF00BF00BF00BF00BF00BF00BF94
:1034400000BF00BF00BF00BF00BF00BFEC63012092
:10345000FCF71AFFB000FCF717FFAC6300BF00BF1A
:1034600000BF00BF00BF00BF00BF00BF00BF00BF64
:1034700000BF00BF00BF00BF00BF00BF00BF00BF54
:1034800000BF00BF00BF00BF00BF00BF00BF00BF44
:1034900000BF00BF00BF00BF00BF00BF70BD2DE96F
:1034A000FE430F46044602A9794800F0BCFD794D61
:1034B000794EDFF8E88148B18220286022207946E1
:1034C00030608220C8F80010BDE8FE839DF8080037
:1034D000800701D4FFF7BCFE02208DF80000200C0D
:1034E0008DF80100200A8DF802008DF803408DF858
:1034F000047000BF00BF00BF00BF00BF00BF00BF1F
:1035000000BF00BF00BF00BF00BF00BF00BF00BFC3
:1035100000BF00BF00BF00BF00BF00BF00BF00BFB3
:1035200000BF00BF00BF00BF00BF00BF00BF00BFA3
:1035300000BF564F4FF48024FC6305216846FCF71A
:10354000AAFEBC6300BF00BF00BF00BF00BF00BF3A
:1035500000BF00BF00BF00BF00BF00BF00BF00BF73
:1035600000BF00BF00BF00BF00BF00BF00BF00BF63
:1035700000BF00BF00BF00BF00BF00BF00BF00BF53
:1035800000BF00BF0020286079463060C8F80010F6
:103590009AE72DE9FC5F3F4D3F4E404F5FEA020A3C
:1035A0008B4604464FF000080DD001A9384800F0C2
:1035B0003AFD80B182202860212030607846386052
:1035C0008220BDE8FC9FC5F800807846C6F80080E0
:1035D00038600020F5E703208DF80000200C8DF8FE
:1035E0000100200A8DF802008DF8034000BF00BFE3
:1035F00000BF00BF00BF00BF00BF00BF00BF00BFD3
:1036000000BF00BF00BF00BF00BF00BF00BF00BFC2
:1036100000BF00BF00BF00BF00BF00BF00BF00BFB2
:1036200000BF00BF00BF00BF00BF00BF174C4FF47A
:103630008029C4F83C9004216846FCF72CFE5146D2
:103640005846FCF734FEC4F8389000BF00BF00BFF6
:1036500000BF00BF00BF00BF00BF00BF00BF00BF72
:1036600000BF00BF00BF00BF00BF00BF00BF00BF62
:1036700000BF00BF00BF00BF00BF00BF00BF00BF52
:1036800000BF00BF00BF00BF00BF9CE700C0092013
:10369000A08601006C000010700000107400001083
:1036A0002DE9F05FFF4EDFF80094DFF800A415006D
:1036B00083460F464FF000080ED000240AE0395D23
:1036C0000BEB0400FFF7EBFE000602D53068BDE807
:1036D000F09F641CAC42F2D3C6F800807946C9F86A
:1036E00000800020CAF80010F1E72DE9FC470446ED
:1036F00001A9EF4800F097FCEA4DEB4EDFF8AC93E0
:1037000048B1822028602220794630608220C9F8A2
:103710000010BDE8FC879DF80400800701D4FFF786
:1037200097FD20208DF8000020098DF80100200170
:103730008DF8020000248DF8034000BF00BF00BFD9
:1037400000BF00BF00BF00BF00BF00BF00BF00BF81
:1037500000BF00BF00BF00BF00BF00BF00BF00BF71
:1037600000BF00BF00BF00BF00BF00BF00BF00BF61
:1037700000BF00BF00BF00BF00BFDFF838834FF4B9
:103780008027C8F83C7004216846FCF784FDC8F81F
:10379000387000BF00BF00BF00BF00BF00BF00BF48
:1037A00000BF00BF00BF00BF00BF00BF00BF00BF21
:1037B00000BF00BF00BF00BF00BF00BF00BF00BF11
:1037C00000BF00BF00BF00BF00BF00BF00BF00BF01
:1037D00000BF2C60794634600020C9F8001098E7DB
:1037E0002DE9FC478A46044601A9B14800F01BFCBC
:1037F000AC4DAD4EDFF8B49240B18220286022205B
:10380000794630608220C9F8001082E703208DF8E5
:10381000000020098DF8010020018DF8020000242D
:103820008DF8034000BF00BF00BF00BF00BF00BF56
:1038300000BF00BF00BF00BF00BF00BF00BF00BF90
:1038400000BF00BF00BF00BF00BF00BF00BF00BF80
:1038500000BF00BF00BF00BF00BF00BF00BF00BF70
:1038600000BF00BFDFF84C824FF48027C8F83C70DF
:1038700004216846FCF70FFDB9115046FCF717FD0F
:10388000C8F8387000BF00BF00BF00BF00BF00BF56
:1038900000BF00BF00BF00BF00BF00BF00BF00BF30
:1038A00000BF00BF00BF00BF00BF00BF00BF00BF20
:1038B00000BF00BF00BF00BF00BF00BF00BF00BF10
:1038C00000BF00BF2C60794634600020C9F80010AA
:1038D0001FE72DE9F34F83B0044601A9744800F0B7
:1038E000A2FB704D704E714F4FF0820818B121202D
:1038F000C5F800806CE09DF80400800701D4FFF754
:10390000A7FCAD208DF8000020098DF801002001F2
:103910008DF802004FF0000B8DF803B000BF00BF20
:1039200000BF00BF00BF00BF00BF00BF00BF00BF9F
:1039300000BF00BF00BF00BF00BF00BF00BF00BF8F
:1039400000BF00BF00BF00BF00BF00BF00BF00BF7F
:1039500000BF00BF00BF00BF00BF00BFDFF8549131
:103960004FF4802A5446C9F83CA004216846FCF76D
:1039700092FC02210498FCF78EFCC9F8384000BF85
:1039800000BF00BF00BF00BF00BF00BF00BF00BF3F
:1039900000BF00BF00BF00BF00BF00BF00BF00BF2F
:1039A00000BF00BF00BF00BF00BF00BF00BF00BF1F
:1039B00000BF00BF00BF00BF00BF00BF00BF0224A8
:1039C00001A93B4800F02FFB48B12220C5F8008038
:1039D000306078463860822005B0BDE8F08F00BFC7
:1039E00000BF00BF00BF00BF00BF00BF00BF00BFDF
:1039F00000BF00BF00BF00BF00BF00BF00BF00BFCF
:103A000000BF00BF00BF00BF00BF00BF00BF00BFBE
:103A100000BF00BF00BF00BF00BF00BF00BFC9F8AC
:103A20003CA0AD20FCF730FC049802212044FCF7B8
:103A300032FCC9F838A000BF00BF00BF00BF00BF04
:103A400000BF00BF00BF00BF00BF00BF00BF00BF7E
:103A500000BF00BF00BF00BF00BF00BF00BF00BF6E
:103A600000BF00BF00BF00BF00BF00BF00BF00BF5E
:103A700000BF00BF00BFA41CA4B2B4F5805F9FD3F9
:103A800001A90B4800F0CFFA00287FF430AFFFF710
:103A900029FCC5F800B07846C6F800B038600020B0
:103AA0009AE700006C000010700000107400001015
:103AB000A086010000C0092070B5FD4DFD4EFE4CF2
:103AC0002AB1FFF766FD000609D5206870BD862083
:103AD00020600920286078463060862070BD002074
:103AE0002060286078463060002070BD2DE9F04FDE
:103AF00089B0DFF8C483DFF8B8B35FEA02094FF09A
:103B0000000607910FD04FF4805501462A466846BB
:103B1000FCF7DCFBDDE90047284601F047F85FEAE7
:103B2000000A0CD016E08621C8F800100921CBF855
:103B300000107946DF480160862009B04DE78221F8
:103B4000C8F800102221CBF800107946D94801604E
:103B50008220F2E7A9EB0605C7F58050A84200D203
:103B60000546B5F5805F04D020465146FFF738FE84
:103B700080B92046FFF7B9FD60B907982A46811938
:103B800007EB0A0001F068F82E4420465146FFF783
:103B9000A0FE28B1504601F038F8D8F80000CCE774
:103BA0000027641C4E45D5D3504601F02EF8002066
:103BB000C8F800007946CBF80000BE48016000203C
:103BC000BBE72DE9FF4F8DB00D46DDF8689000266C
:103BD000B94C07935FEA09013FD04FF48057014683
:103BE0003A466846FCF772FBDDE900B10C913A46B3
:103BF000691C6846FCF76AFBDDE90010CDE90401A9
:103C00003A4668460F99FCF761FBDDE9008500BF85
:103C1000A9EB0607C5F58050B84200D2074625B18A
:103C2000D8457CD10C98854279D14FF4805000F072
:103C3000BDFF5FEA000A1BD0D8454FD10C988542E2
:103C40004CD12A464FEA08305146FFF7A2FC000645
:103C500018D5504600F0D9FF79E0862020609448BE
:103C600009210160784693490860862011B0B4E6C6
:103C7000822020608E482221016079468D480160B3
:103C80008220F3E70598804509D1049901EB0030C3
:103C9000C1F580525144FFF77CFC0006D9D4404660
:103CA000FFF723FD0006D4D407983A46811905EBA7
:103CB0000A0000F0D1FFEA194FEA08305146FFF739
:103CC000EFFC0006C5D40599884533D1049800EB74
:103CD00001300499C1F58052514427E00599884587
:103CE0000AD1049800EB01300499C1F58052514685
:103CF000FFF74FFC0006ACD44046FFF7F6FC000689
:103D0000A7D407983A4681190F983044FFF7C8FCAA
:103D100000069ED4059988450CD1049800E00DE07A
:103D200000EB01300499C1F580525146FFF7B8FC11
:103D300000068ED4504600F068FF0AE007983A4625
:103D400081190F983044FFF7ABFC000601D52068BD
:103D50008CE73E44002508F101084E45FFF458AFBA
:103D600053490020206008607846524908600020CE
:103D70007CE72DE9F0474FF0000900BF00BF00BF0E
:103D800000BF00BF00BF00BF00BF00BF00BF00BF3B
:103D900000BF00BF00BF00BF00BF00BF00BF00BF2B
:103DA00000BF00BF00BF00BF00BF00BF00BF00BF1B
:103DB00000BF00BF00BF00BF00BF404E4FF48025D2
:103DC000F5639F20FCF760FA0020FCF75DFA00F035
:103DD000FF080020FCF758FAC4B20020FCF754FAA0
:103DE000C1B2B56300BF00BF00BF00BF00BF00BFCE
:103DF00000BF00BF00BF00BF00BF00BF00BF00BFCB
:103E000000BF00BF00BF00BF00BF00BF00BF00BFBA
:103E100000BF00BF00BF00BF00BF00BF00BF00BFAA
:103E200000BF00BF244D224E224FB8F1BF0F03D177
:103E3000252C0AD0262C08D0822028602120306032
:103E4000784638608220BDE8F0871D48412912D0AD
:103E50004FF48002422912D04A2910D0C0F80090B5
:103E60000020FFF789FAC5F800907846C6F8009060
:103E700038600020E7E74FF400110160F0E70260CE
:103E8000EEE72DE9F84F69460E4800F0CCF882279E
:103E9000094C074D074E4FF0220A002862D19DF8C9
:103EA0000000800701D4FFF7D3F900BF00BF0BE08B
:103EB00070000010740000106C00001000C0092099
:103EC00018010010A086010000BF00BF00BF00BFA6
:103ED00000BF00BF00BF00BF00BF00BF00BF00BFEA
:103EE00000BF00BF00BF00BF00BF00BF00BF00BFDA
:103EF00000BF00BF00BF00BF00BF00BF00BF00BFCA
:103F000000BF00BFDFF8EC914FF48028C9F83C8077
:103F10006020FCF7B9F9C9F8388000BF00BF00BFC6
:103F200000BF00BF00BF00BF00BF00BF00BF00BF99
:103F300000BF00BF00BF00BF00BF00BF00BF00BF89
:103F400000BF00BF00BF00BF00BF00BF00BF00BF79
:103F500000BF00BF00BF00BF00BF6946664800F059
:103F600062F838B127607846C5F800A0306082203A
:103F7000BDE8F88F0020206028607846306000207F
:103F8000F6E75E48006870474FF4805070472DE9AF
:103F9000F04FDFF86C81DFF86CB189B00F00044698
:103FA0004FF0000626D04FF4805501462A46684659
:103FB000FCF78CF9DDE900A105912A46214606A807
:103FC000FCF784F9DDE906404FF00009BD1BC0F5A0
:103FD0008051A94200D20D4620B1544515D1059912
:103FE000884212D12046FFF780FB00060DD5D8F895
:103FF0000000A2E58621C8F800100921CBF80010C6
:10400000794641480160862097E52E44641C484665
:10401000BE42DBD3C8F800007946CBF800003A482E
:104020000160002089E52DE9F041384C0F46064635
:10403000A56806E0A068401BB04202D30120BDE89D
:10404000F081384600F003F80028F3D1F7E770B5A7
:10405000044600BF00BF00BF00BF00BF00BF00BFDD
:1040600000BF00BF00BF00BF00BF00BF00BF00BF58
:1040700000BF00BF00BF00BF00BF00BF00BF00BF48
:1040800000BF00BF00BF00BF00BF00BF00BF00BF38
:1040900000BF184E4FF48025F5630520FCF7F4F8B7
:1040A0000020FCF7F1F82070B56300BF00BF00BF2F
:1040B00000BF00BF00BF00BF00BF00BF00BF00BF08
:1040C00000BF00BF00BF00BF00BF00BF00BF00BFF8
:1040D00000BF00BF00BF00BF00BF00BF00BF00BFE8
:1040E00000BF00BF00BF00BF00BF207800F001008C
:1040F00070BD000000C0092020A1070018010010B9
:104100006C000010700000107400001000000940E6
:104110002DE9FF4703A9FE4800F063FBFD4DFE4E6D
:10412000DFF8F89350B18220286021207946306072
:104130008220C9F8001004B0BDE8F0879DF80C009B
:10414000800701D4FFF784F842208DF80000002496
:10415000CDF80140CDF80540ADF8094000BF00BFE3
:1041600000BF00BF00BF00BF00BF00BF00BF00BF57
:1041700000BF00BF00BF00BF00BF00BF00BF00BF47
:1041800000BF00BF00BF00BF00BF00BF00BF00BF37
:1041900000BF00BF00BF00BF00BF00BFDFF88083CB
:1041A0004FF48027C8F83C700B216846FCF773F881
:1041B000C8F8387000BF00BF00BF00BF00BF00BF1D
:1041C00000BF00BF00BF00BF00BF00BF00BF00BFF7
:1041D00000BF00BF00BF00BF00BF00BF00BF00BFE7
:1041E00000BF00BF00BF00BF00BF00BF00BF00BFD7
:1041F00000BF00BF2C60794634600020C9F8001071
:1042000099E72DE9F34F85B0044603A9C04800F0B3
:10421000E8FAC04DC04EC14F4FF0820B18B12120BB
:10422000C5F800B060E0FFF713F842208DF80000F9
:104230004FF0000ACDF801A0CDF805A0ADF809A017
:1042400000BF00BF00BF00BF00BF00BF00BF00BF76
:1042500000BF00BF00BF00BF00BF00BF00BF00BF66
:1042600000BF00BF00BF00BF00BF00BF00BF00BF56
:1042700000BF00BF00BF00BF00BF00BF00BF00BF46
:10428000DFF89C924FF48028C9F83C800B216846E7
:10429000FCF701F8C9F8388000BF00BF00BF00BFBD
:1042A00000BF00BF00BF00BF00BF00BF00BF00BF16
:1042B00000BF00BF00BF00BF00BF00BF00BF00BF06
:1042C00000BF00BF00BF00BF00BF00BF00BF00BFF6
:1042D00000BF00BF00BF00BF03A98D4800F081FAF6
:1042E00048B12220C5F800B030607846386082209E
:1042F00007B0BDE8F08F9DF80C00800701D4FEF7F1
:10430000A7FF02208DF80000200C8DF80100200A84
:104310008DF8020006988DF803408DF8040000BF68
:1043200000BF00BF00BF00BF00BF00BF00BF00BF95
:1043300000BF00BF00BF00BF00BF00BF00BF00BF85
:1043400000BF00BF00BF00BF00BF00BF00BF00BF75
:1043500000BF00BF00BF00BF00BF00BF00BF44469A
:10436000C846C9F83C4005216846FBF794FFC8F8E9
:10437000384000BF00BF00BF00BF00BF00BF00BF8C
:1043800000BF00BF00BF00BF00BF00BF00BF00BF35
:1043900000BF00BF00BF00BF00BF00BF00BF00BF25
:1043A00000BF00BF00BF00BF00BF00BF00BF00BF15
:1043B00000BFC5F800A07846C6F800A0386000200D
:1043C00096E72DE9F05F534EDFF84C91DFF84CA1F2
:1043D000150083460F464FF000080ED000240AE077
:1043E000395D0BEB0400FFF70CFF000602D53068C7
:1043F000BDE8F09F641CAC42F2D3C6F80080794659
:10440000C9F800800020CAF80010F1E72DE9F34F49
:104410000024404D404E414FC3B080464FF0820AC9
:104420004FF0210BA14641A9394800F0DAF90028E4
:104430007CD19DF80401800701D4FEF709FF02201A
:104440008DF800004FEA18108DF8010004EB0810F9
:104450008DF8020044988DF8039000EB04214FF48E
:10446000807201A800F0F8FB00BF00BF00BF00BFD2
:1044700000BF00BF00BF00BF00BF00BF00BF00BF44
:1044800000BF00BF00BF00BF00BF00BF00BF00BF34
:1044900000BF00BF00BF00BF00BF00BF00BF00BF24
:1044A00000BF00BF00BF00BF1D494FF48020C8639C
:1044B0004FF482716846FBF7EEFE19494FF48020F5
:1044C000886300BF00BF00BF00BF00BF00BF00BFC8
:1044D00000BF00BF00BF00BF00BF00BF00BF00BFE4
:1044E00000BF00BF00BF00BF00BF00BF00BF00BFD4
:1044F00000BF00BF00BF00BF00BF00BF00BF00BFC4
:1045000000BF641CE4B2102C8DD341A900480AE01E
:10451000A08601006C0000107000001074000010F4
:1045200000C0092002E000F05CF940B1C5F800A02D
:104530007846C6F800B03860822045B0D9E6FEF76C
:10454000D1FEC5F800907846C6F80090386000208B
:10455000F3E72DE9F04F89B0DFF85483DFF854B367
:104560005FEA02094FF0000607910FD04FF4805523
:1045700001462A466846FBF7A9FEDDE900472846C2
:1045800000F014FB5FEA000A0CD016E08621C8F8A0
:1045900000100921CBF800107946C7480160862039
:1045A00009B0A6E68221C8F800102221CBF800103D
:1045B0007946C14801608220F2E7A9EB0605C7F5FC
:1045C0008050A84200D20546B5F5805F04D0204651
:1045D0005146FFF705F980B92046FFF786F860B924
:1045E00007982A46811907EB0A0000F035FB2E4494
:1045F00020465146FFF70AFF28B1504600F005FB60
:10460000D8F80000CCE70027641C4E45D5D35046AF
:1046100000F0FBFA0020C8F800007946CBF8000053
:10462000A54801600020BBE72DE9FF4F8DB00D4686
:10463000DDF8689000269E4C07935FEA09013ED0A2
:104640004FF4805701463A466846FBF73FFEDDE9E6
:1046500000B10C913A46691C6846FBF737FEDDE96C
:104660000010CDE904013A4668460F99FBF72EFE8B
:10467000DDE90085A9EB0607C5F58050B84200D2F8
:10468000074625B1D8457CD10C98854279D14FF4A5
:10469000805000F08BFA5FEA000A1BD0D8454FD15A
:1046A0000C9885424CD12A464FEA08305146FEF715
:1046B00070FF000618D5504600F0A7FA79E0862072
:1046C00020607C480921016078467B49086086208B
:1046D00011B00EE6822020607648222101607946E2
:1046E000754801608220F3E70598804509D1049957
:1046F00001EB0030C1F580525144FEF74AFF00063D
:10470000D9D44046FEF7F1FF0006D4D407983A46C4
:10471000811905EB0A0000F09FFAEA194FEA083008
:104720005146FFF74EFE0006C5D40599884533D1A2
:10473000049800EB01300499C1F58052514427E000
:10474000059988450AD1049800EB01300499C1F518
:1047500080525146FEF71DFF0006ACD44046FEF7DE
:10476000C4FF0006A7D407983A4681190F98304431
:10477000FFF727FE00069ED4059988450CD10498C2
:1047800000E00DE000EB01300499C1F58052514684
:10479000FFF717FE00068ED4504600F036FA0AE006
:1047A00007983A4681190F983044FFF70AFE000631
:1047B00001D520688CE73E44002508F101084E45EC
:1047C000FFF458AF3B4900202060086078463A4922
:1047D000086000207CE74FF4800070474FF4805061
:1047E00070472DE9F041354C0F460646A56806E0B6
:1047F000A068401BB04202D30120BDE8F0813846DA
:1048000000F003F80028F3D1F7E770B5044600BFC5
:1048100000BF00BF00BF00BF00BF00BF00BF00BFA0
:1048200000BF00BF00BF00BF00BF00BF00BF00BF90
:1048300000BF00BF00BF00BF00BF00BF00BF00BF80
:1048400000BF00BF00BF00BF00BF00BF00BF1C4EC5
:104850004FF48025F5630520FBF716FD0020FBF7DC
:1048600013FD2070B56300BF00BF00BF00BF00BFD5
:1048700000BF00BF00BF00BF00BF00BF00BF00BF40
:1048800000BF00BF00BF00BF00BF00BF00BF00BF30
:1048900000BF00BF00BF00BF00BF00BF00BF00BF20
:1048A00000BF00BF00BF207800F0010070BD000015
:1048B0006C0000107000001074000010000009402F
:1048C00000C0092000207047AE4982200860AE4930
:1048D000212008607846AD49086082207047A949C8
:1048E00082200860A849222008607846A74908600D
:1048F00082207047A34982200860A34922200860D3
:104900007846A24908608220704770B5002400BF35
:1049100000BF00BF00BF00BF00BF00BF00BF00BF9F
:1049200000BF00BF00BF00BF00BF00BF00BF00BF8F
:1049300000BF00BF00BF00BF00BF00BF00BF00BF7F
:1049400000BF00BF00BF00BF00BF00BF00BF904E50
:104950004FF48025F5639F20FBF796FC0020FBF7C2
:1049600093FC60F307040020FBF78EFC60F30F2438
:104970000020FBF789FC60F31744B56300BF00BF5C
:1049800000BF00BF00BF00BF00BF00BF00BF00BF2F
:1049900000BF00BF00BF00BF00BF00BF00BF00BF1F
:1049A00000BF00BF00BF00BF00BF00BF00BF00BF0F
:1049B00000BF00BF00BF00BF00BF00BF7549601A45
:1049C0008C421AD00BDCA4F1C204B4F5A11414D0AB
:1049D000B4F5803F11D0B4F5003F0BD10DE06E4926
:1049E000401805D06D49401809D06D49C84201D121
:1049F000022400E00024204670BD0324FBE70424C9
:104A0000FFF786FBF7E76748007828B1664900EBB7
:104A1000C00051F8200000475A49822008605A49D6
:104A2000212008607846594908608220704770B597
:104A3000FFF76BFF5B49544D544E524C087050B118
:104A4000594900EBC00001EB8000806880470006F8
:104A500009D5206870BD822020602120286078461A
:104A60003060822070BD0020206028607846306071
:104A7000002070BD2DE9F0414A4B434D434E1B7859
:104A8000404C63B19AB1484F03EBC30307EB830378
:104A90001B699847000612D52068BDE8F081822086
:104AA000206021202860784630608220F5E786204B
:104AB000206009202860784630608620EDE70020DD
:104AC00020602860784630600020E6E72DE9F0415C
:104AD000344B2D4D2D4E1B782A4C5BB192B1324F89
:104AE00003EBC30307EB83039B699847000611D5CB
:104AF0002068D2E78220206022202860784630603B
:104B00008220CAE78620206009202860784630602D
:104B10008620C2E7002020602860784630600020B0
:104B2000BBE7F8B51F4C184D184E2778154CDDF82B
:104B300018C087B1BCF1000F15D0CDF800C0DFF868
:104B400068C007EBC7070CEB8707FF69B84700068B
:104B500011D52068F8BD8220206022202860784688
:104B600030608220F8BD86202060092028607846C9
:104B700030608620F8BD00202060286078463060D4
:104B80000020F8BD6C0000107000001074000010D0
:104B900000C00920C220180003FBD6FF00FFFEFF63
:104BA0000001F8FF1C010010F453000070B5064628
:104BB000FBF79AFB056806F10B0020F00704B442EE
:104BC0009CBF002070BD2B466A68BAB11068A04235
:104BD00010D304F1080188423CBF5068586007D3E5
:104BE0005168101941601168091B01605860146018
:104BF000101D70BD13465268002AE7D12146284691
:104C000000F0A3F80028DED170BD70B50446051F82
:104C1000FBF76AFB0068002C14BF446870BD002CD1
:104C200018BFAC423CBF20466468F8D301680A183C
:104C3000AA4218BF456003D12A68054611440160A5
:104C400028684119A1421CBF6C6070BD6168696031
:104C500021680844286070BD032A40F2308010F0BB
:104C6000030C00F0158011F8013BBCF1020F624407
:104C700098BF11F801CB00F8013B38BF11F8013B98
:104C8000A2F1040298BF00F801CB38BF00F8013B45
:104C900011F0030300F02580083AC0F0088051F8B5
:104CA000043B083A51F804CBA0E80810F5E7121DC0
:104CB0005CBF51F8043B40F8043BAFF30080D207DF
:104CC00024BF11F8013B11F801CB48BF11F8012BAB
:104CD00024BF00F8013B00F801CB48BF00F8012BCE
:104CE000704710B5203AC0F00B80B1E81850203A58
:104CF000A0E81850B1E81850A0E81850BFF4F5AF7C
:104D00005FEA027C24BFB1E81850A0E8185044BF05
:104D100018C918C0BDE810405FEA827C24BF51F872
:104D2000043B40F8043B08BF7047D20728BF31F866
:104D3000023B48BF11F8012B28BF20F8023B48BFB7
:104D400000F8012B70477047704738B504460A4693
:104D500000206946AFF30080002808BF38BD024636
:104D600000992046FBF72FFB012038BD012000F001
:104D70002FB8F8B5AFF30080054600200C46102090
:104D800000BF0646A819A0420DD932466946002048
:104D9000AFF30080070008BF00F01AF80098A042A7
:104DA00018BF0546C419FBF79FFA05600746F01DBA
:104DB00020F0070046192846FBF7FEFAB44208BF68
:104DC000F8BDA21B31463868BDE8F840FBF7FBBAD6
:104DD00010B500F037F8BDE8104000F02EB8754669
:104DE000FBF788FAAE4605006946534620F00700F7
:104DF000854618B020B5FBF7EFF9BDE820404FF02D
:104E000000064FF000074FF000084FF0000B21F0B4
:104E10000701AC46ACE8C009ACE8C009ACE8C00981
:104E2000ACE8C0098D46704710B50446AFF300806A
:104E30002046BDE81040FBF794B9002801D000F0EF
:104E400029B8704710B5012805D0002103A000F053
:104E500027F8012010BD09A1F8E700005349475287
:104E6000544D454D3A204F7574206F66206865613A
:104E700070206D656D6F7279000000003A20486502
:104E80006170206D656D6F727920636F72727570DD
:104E90007465640001491820ABBEFEE726000200DD
:104EA00070B505460C460A2000E06D1C00F011F8B4
:104EB00035B128780028F8D102E0641C00F009F828
:104EC00014B120780028F8D1BDE870400A20AFF373
:104ED000008008B569468DF800000320ABBE08BD10
:104EE00000050F0A1B1E141133363C39282D2722CA
:104EF00063666C69787D777250555F5A4B4E4441BA
:104F0000C3C6CCC9D8DDD7D2F0F5FFFAEBEEE4E1A9
:104F1000A0A5AFAABBBEB4B193969C99888D878299
:104F200083868C89989D9792B0B5BFBAABAEA4A189
:104F3000E0E5EFEAFBFEF4F1D3D6DCD9C8CDC7C279
:104F400040454F4A5B5E545173767C79686D676269
:104F500023262C29383D373210151F1A0B0E040159
:104F600003060C09181D171230353F3A2B2E242149
:104F700060656F6A7B7E747153565C59484D474239
:104F8000C0C5CFCADBDED4D1F3F6FCF9E8EDE7E229
:104F9000A3A6ACA9B8BDB7B290959F9A8B8E848119
:104FA00080858F8A9B9E9491B3B6BCB9A8ADA7A209
:104FB000E3E6ECE9F8FDF7F2D0D5DFDACBCEC4C1F9
:104FC00043464C49585D575270757F7A6B6E6461E9
:104FD00020252F2A3B3E343113161C19080D0702D9
:104FE00000002110422063308440A550C660E77065
:104FF000088129914AA16BB18CC1ADD1CEE1EFF10D
:105000003112100273325222B5529442F772D662B4
:10501000399318837BB35AA3BDD39CC3FFF3DEE35C
:105020006224433420040114E664C774A444855404
:105030006AA54BB528850995EEE5CFF5ACC58DD5AC
:105040005336722611163006D776F6669556B44654
:105050005BB77AA719973887DFF7FEE79DD7BCC7FC
:10506000C448E5588668A7784008611802282338A4
:10507000CCC9EDD98EE9AFF9488969990AA92BB94C
:10508000F55AD44AB77A966A711A500A333A122AF4
:10509000FDDBDCCBBFFB9EEB799B588B3BBB1AAB9C
:1050A000A66C877CE44CC55C222C033C600C411C44
:1050B000AEED8FFDECCDCDDD2AAD0BBD688D499DEC
:1050C000977EB66ED55EF44E133E322E511E700E94
:1050D0009FFFBEEFDDDFFCCF1BBF3AAF599F788F3C
:1050E0008891A981CAB1EBA10CD12DC14EF16FE11C
:1050F0008010A100C230E320045025404670676054
:10510000B9839893FBA3DAB33DC31CD37FE35EF36B
:10511000B1029012F322D2323542145277625672A3
:10512000EAB5CBA5A89589856EF54FE52CD50DC5BB
:10513000E234C324A01481046674476424540544F3
:10514000DBA7FAB79987B8975FE77EF71DC73CD70B
:10515000D326F2369106B016576676761546345643
:105160004CD96DC90EF92FE9C899E9898AB9ABA95B
:105170004458654806782768C018E1088238A32893
:105180007DCB5CDB3FEB1EFBF98BD89BBBAB9ABBAB
:10519000754A545A376A167AF10AD01AB32A923AE3
:1051A0002EFD0FED6CDD4DCDAABD8BADE89DC98DFB
:1051B000267C076C645C454CA23C832CE01CC10C33
:1051C0001FEF3EFF5DCF7CDF9BAFBABFD98FF89F4B
:1051D000176E367E554E745E932EB23ED10EF01E83
:1051E000EB3C904D53444F53352E300002020100EA
:1051F0000110000004F80C00010001000000000094
:1052000000000000000029EFBEADDE41544F4C20ED
:10521000465072696E74464154313220202000009D
:10522000000000000010000000200000003000001E
:10523000004000000050000000600000007000000E
:10524000008000000090000000A0000000B00000FE
:1052500000C0000000D0000000E0000000F00000EE
:105260000000010000800100000002000080020038
:105270000000030000800300000004000080040020
:105280000000050000800500000006000080060008
:105290000000070000800700FF0F0000FF1F000054
:1052A000FF2F0000FF3F0000FF4F0000FF5F0000E6
:1052B000FF6F0000FF7F0000FF8F0000FF9F0000D6
:1052C000FFAF0000FFBF0000FFCF0000FFDF0000C6
:1052D000FFEF0000FFFF0000FF7F0100FFFF010064
:1052E000FF7F0200FFFF0200FF7F0300FFFF0300BC
:1052F000FF7F0400FFFF0400FF7F0500FFFF0500A4
:10530000FF7F0600FFFF0600FF7F0700FFFF07008B
:10531000120110010000004051C2031300010420DB
:105320004801090220000101008032090400000246
:10533000080650620705820240000007050202408D
:10534000000000040309041C03410054004F004CFA
:10535000002000200020002000200020002000204D
:10536000002000280346005000720069006E00749F
:1053700000200046006C00610073006800200020DF
:1053800000200020002000200020001A03460069B1
:105390000072006D0077006100720065003000301F
:1053A00000300030000E034D0065006D006F00728C
:1053B00000790000F12300000000000093030000CA
:1053C00000000000000000000000000000000000DD
:1053D00000000000000000000000000000000000CD
:1053E00000000000000000000000000000000000BD
:1053F00000000000C5480000C5480000C948000082
:10540000DF480000C9480000DF480000DF48000016
:10541000DF480000F5480000C5480000C54800000E
:10542000C9480000DF480000C9480000DF4800000C
:10543000DF480000DF480000F5480000833F00001F
:10544000893F0000733D0000833E0000B93A000030
:10545000ED3A0000A1360000C33B00008F3F000082
:10546000BB300000C1300000BD2B0000833E0000B7
:10547000B93A0000172E0000C34300000B2F0000B4
:10548000C7300000D7470000DD470000733D000033
:10549000833E0000B93A000053450000C3430000BA
:1054A000294600008F3F00000000000000000000BF
:1054B00000000000000000000000000000000000EC
:1054C000000000000000000000000000EC5400009C
:1054D0000000001020010000080100000C56000030
:1054E00020010010607000002401000041544F4C66
:1054F00020465072696E7428000000000000000011
:105500000000D4284B3D0000000000000000000017
:10551000000000000000000000000000000000008B
:10552000000000000000000000000000000000007B
:10553000000000000000000000000000000000006B
:10554000000000000000000000000000000000104B
:10555000000000000000000000000000000000004B
:10556000000000000000000000000000000000003B
:10557000000000000000000000000000000000002B
:10558000000000000000000000000000000000001B
:10559000000000000000000000000000000000000B
:1055A00000000000000000000000000000000000FB
:1055B00000000000000000000000000000000000EB
:1055C0000000000000093D00000000000000000095
:1055D00000000000000000000000000000000000CB
:1055E00000000000000000000000000000000000BB
:1055F00000000000000000000000000000000000AB
:105600000000000000000000000000000588C270DB
:1056100080A487165401FD65D8FF1F5CF79517D548
:105620002F2FD2A84BFD9D12C67F8D8DB6EA2C0E72
:10563000F4144DE1038D36EFCEFE55B0AE3E325B35
:105640006943BF72DE080452200CFED06772E9F78E
:10565000C67CCA977D4E0F27766AEDC7D36CD8A457
:10566000C9CAA8B3CA84E8857C2C1EFD2649F34626
:105670007F8F14186D1784948AAF487E4CFBBD76DB
:105680006BC47731EBAE60AECCABEFCE9CA3132FE7
:10569000B2DD09CFF06B35428AF2A4E8A34B49444E
:1056A000E449F80BBC349EF4120DAF24319688F413
:1056B00095E87DB36FDA7398D4B374CE3E67DF6735
:1056C0004E1DEE418C3FAA450A5528EBD5A4658AAC
:1056D000F64515294CE102E3D72E0111710ACB7969
:1056E0000D5D6EA02BB37FE26F046428F07CF3E0C5
:1056F000B077B1EB47DB26C14840991DDF27700F1B
:105700005D4F80EC14068697E3BFFE28FB8ECB78B6
:10571000A4DF782F951E61BDA09525BB15464A5F75
:1057200041C1BBC01EB24D25E8FAAAD5B3584169A4
:10573000DE648D54ACFE61D53BB4F7CFF94C2173D8
:10574000F8D8B7FF817495DEC2068069B432F26181
:105750006B4FED3E4FA3FCF2C15F8F27995EFA4A73
:105760002E92E26290821DD65C639A3F8903DB2908
:10577000C005A2638D1BEB70C441CC8353176ED65A
:1057800050B82A719308E202E8BC3E6C041EA340A4
:105790006716CF1B317EE4092C4898E5C82B245DA1
:1057A000D89447D3E8CCE8300631035754261895EF
:1057B000F1909729E4F9EBE57611D813E6D7971421
:1057C000AA7F8B28C0DF8766670366BE4A9F43F9BE
:1057D000A10E25136A67A9C7BF56D29631EDCE0B2D
:1057E0006EC693B285F3044B3863FC21FBCB54EDBA
:1057F000B01F7384ED7FF96562654896DBDE416C0E
:10580000CB7F22EA03076717D8E674F9F1E13E5F20
:10581000C9C0F87003EDE4CC4F2C753A4904277CDD
:105820002698022A51D71E2AB01C4AEBD20D144CDE
:10583000DD9B9CA323AACAF08083310453FA8AD249
:105840005F253FEA9A87AF3ABFC19E306D96B3ABF2
:10585000FBE264B987738C38B8007E88F7CFFF12FB
:105860007E641C5A59F5BC941BDF7FB9766D656365
:10587000B2AFDE82B40F40C9429A8D10A28716687B
:10588000E977C7A77B4F4C287D6561DC1FC45F9318
:10589000E00CE5FA52E976A06E6B1D500FAEA997A9
:1058A00032DA2657215DDB6A829179C273FCF05FA0
:1058B00053B78B37A8E9749D5F256A447E5BE6A5E4
:1058C000BBAB5C9F9E018EC1C7F9B5699A3126DCDE
:1058D00089B231F149CE7D185EC80E58867DC99CCB
:1058E000A80C5D13D57A6AF4D9238E35C918F4460D
:1058F000D7A18CE2E9640C7044B08A4EC8A1781F2D
:105900003418BED38104DADF1E56499FE0F47C4C84
:10591000542548842A54E7B07C7800FFC1F7F4830B
:1059200076CD001A291D32DEA6BDA1B1826B564F7D
:10593000DB598780E5F209166D5B4D8164706DE27D
:1059400057DA0C8E7B67B87DD8CAFB35AFD3128E81
:10595000E5796A7CD7D9858E8320234DDB97D1FBEF
:10596000CF3CE0878C095C3E7ACDEB2867937ECEF6
:10597000D84541D18F01D41A1717E0FA25F8294EDE
:10598000FB58F051AADCB9D13A5D823366D376DC9C
:10599000D96400FAC9BF0D42DB413DAE18A4B6354B
:1059A0002B37354D14FEF67F91158AA2D19770954D
:1059B000069F3DB29D1B7D9C81B73C787E8BE6F5B2
:1059C0003A69E04DD897E175FD9E5E1CAD3CBE98EE
:1059D0000CBC80F21635A2AFFB79B18F4E66B4F8DD
:1059E000383A16C1400C0A5C9EED3EEE95D229A0D5
:1059F000A6052ED781596B446E4C3281E8C1F37AEB
:105A000086D4C4B9535052CDD7B8F1DB492126C84A
:105A10001D4202B37705CF8FE3168BC4881A9A9381
:105A2000CEA9A778C5BE2B403E0AEE60F4A98CB87B
:105A3000398A3F7408735FE286DD3848D66A4D6B59
:105A40006A498570D28C706F75A5374F83434D3D81
:105A5000696EB7D6144BCE5ACD72663FC6756CD2FE
:105A6000D849EAD0FF8DE05BBFE79926033821646F
:105A700044ABDBB41612310B306B6266AA31F80B03
:105A80004ADC1C0DDFE93BF1F5EE3E9DF133010AE6
:105A9000C9F8E350ECB2EF947B96635FD512BEB7C2
:105AA00095A132DC0E81A0B4CC2D320E91A8865C7B
:105AB0002407483655A28A8C5EA8181E3AA0C54015
:105AC0002063163EA1B62660F6E8D89B72BA391359
:105AD000B96BE9773C84C1259085747E3C1681477B
:105AE000631E2071FC397A93005DDE1692816C276B
:105AF00046E6F12E120B76125EF292E7BE7D885ECC
:105B000096060B49ED04CD7A05FE0EAFCFB238965E
:105B10005027C8E5B4578F77B787289CE3EA90F9F8
:105B200072D52B6B735812AEAA65AE5956F0322857
:105B30005D5674B977F3CEE0B8DF9C30A7B80D5A44
:105B4000F04EC53FDB727454A1F47A5AE823AB17C8
:105B5000B580FF2401B35201B38896102D3B3BC79B
:105B600081D120D991411B9FC956E27DEB68878581
:105B7000A6A5F87BFC6B74004732E9D648B5DEF584
:105B8000CFEC0FDE14597DAD94D3205F1F3FAEC123
:105B90002A239B91B9FDA154B2B836EB2EE3E0D194
:105BA000B80554DF3B519A06EB4F82E90DEB5FDB02
:105BB000454ADCBCED0EE3B72B42CE59F2FDC0E501
:105BC00075C900D995034E58173E2F7228F3DDECA6
:105BD0009A094E92C6CFE0159F6ECFD4B5DBE41183
:105BE000B5FC76720876199AD6C39368B6859C334D
:105BF0003373CD8E65BF1D7DFDB936C5C95F54A316
:105C00003083BE32CFAA7F3C4E2079C50DD9B69CD9
:105C100088A8DC9602583B12DF5441773F5B4FF572
:105C2000430F28D21F2FAD499850619927BEB22843
:105C3000BF1D334B0FC00A9EC9749C21CA860F0C2E
:105C40005200B4AF2CA60A237308628D6C8BC56B0F
:105C50009CFF31FE804605F3AEC09C3CFB37F4EE62
:105C60007910A98CCC39C9129081315A333C20FB70
:105C7000745F097339283013ABD0B2033D09546106
:105C8000F73F5E5B74CED26431BE779C8B93E18725
:105C9000AA64FDF1669644C1A0FA5623EF9E5DBA50
:105CA000FA0600BDA6E8C3318F9836CE5F44A1F650
:105CB000FB7CBAF99C4DBE601394AE2ADED925E96F
:105CC000ADF0B7241A25FD86DBC42481BB4AA42B82
:105CD00055B0194E21555E02AA0252FC93886145C7
:105CE000DC31736B86BD9F25226DBC682B66E3C2D9
:105CF00095BB022FDB9A35E0E564883FF7A6921743
:105D0000CF83B73BAC279B8957C1B8C9A080A39A62
:105D1000F7A15DF9C033F3E5D342EF589F6265D335
:105D2000EEBDE14D4DDAD936D4518E3027E130C683
:105D3000EEF070C0349225B546806A84A83B867622
:105D400058ADC8AA213B65BE18BE0A4FE4F1BA9906
:105D50005663E4524A2B1E6A556FE33BCD1BCD4C74
:105D60000D686FF114977C8E9CB13989D2F9198A2C
:105D700068AF569AF7F9E97DA266568F1B836F7C50
:105D8000542A42AA0DA73DD27E6BE4D41B4AE40FED
:105D9000D8CD2027D1380935E7365CAEA67320EB85
:105DA000977F49B2D9B362308D826B523939EAC4D8
:105DB0006AD89D106718A8610F0AFB7979B95C470A
:105DC0004A9A91F20BC4F2B215C4250FF62430A4FE
:105DD000625CD09A70D34A5BE6F8A70C9531A7D7DE
:105DE0009D9FC1FB4ABE9C7BF698F478E2EE4A1375
:105DF000BB8A8EF8E4575EC05F0CDDB9DC1E75709F
:105E0000D771B12FBDF037B36A03A66592A765AF0E
:105E10002FB339C7C98D495137FBF367CFD1083844
:105E2000DAE36B8C1ACC365508A080A5FFFD0AE298
:105E300034672AD170F2596B8F19ED3A5954416584
:105E4000B70D651613CD0516CCDDB5C748FFB93FB4
:105E50006B4ECEFF238C6E776E2BD62F61BA003936
:105E6000CEAFEBF2D57E81CE222D81A0B851E2CF0C
:105E7000A7E93DAFB5F73748A9E5C6FE8884E051EC
:105E8000444B22A7FE8CFB6613A70E89D444E50F72
:105E90008DEA8E0D0E2045E11706F7F802333A32EF
:105EA0007AA71D0D7626378FA1D8A7F2702E44B69B
:105EB000A017D6C66576B5B70C0A180FA5F693FAE3
:105EC0000F46563596D77B427FF3C717235B52E8C0
:105ED000042DBD28B12890E118BF6F1C0E87D10C8E
:105EE000F68AFA16006BA9F4A8CF96C2B05A191A0E
:105EF000B1DAFF3AC1489A89FE3F3857E61BF0F104
:105F0000033452BD7BD9D957A8C1B6DF677757EDA7
:105F10006C7CFAA013C1715196743FBDEA8AE814F3
:105F2000F88EDDDDEFD1B5FE2AB5862479CDD025FA
:105F3000A7E3FC0FE53AA0AFD23F133B45BC70A2EC
:105F4000CB911F905E75F051B5613075877021312E
:105F50008FAAFBD09888BC54B82E73E4CD096C3D51
:105F6000E550D4C6F5C615EC7EE340BA73736F2BCB
:105F7000303CE8D492C70E2BFA1C3AE91E3E711B46
:105F80003ACA6B4F82C996F81C0DAA0C469F720C38
:105F900049B5C279AAB6ABC375A3272CB37189885A
:105FA00026DD60067356F7096B5A6A6F424DFEEAAA
:105FB000CF06605A9FA5001214DED0D0B936569F86
:105FC0005A043766488117568AB5A2E1EA26D020DE
:105FD000297928D535425332BDA466A7196708D15F
:105FE0004DAD5BE2F4E109B90CAE9AB85A2A22F041
:105FF0009D57482717C975F7D9FD5EFE5199789DC1
:00000001FF
